:020000040000FA
:10000000C0B6D1C0C1C4CCEC0000000000000000AC
:1000100000000000030000000002000014000000C7
:100020000160704743F6C76CC0F60D0C604745F29F
:10003000832CC0F6020C604748F2255CC0F60C0C1D
:10004000604741F29B6CC0F60E0C604745F2E91C1C
:10005000C0F6020C604745F29D2CC0F60D0C6047BF
:1000600041F6195CC0F60D0C604745F2F73CC0F64E
:100070000D0C604744F6416CC0F60D0C604741F230
:10008000CF5CC0F60E0C604745F6992CC0F60D0CFF
:10009000604742F2696CC0F60D0C604742F2C76CD3
:1000A000C0F60D0C604741F6110CC0F60D0C604710
:1000B0004DF63D2CC0F60C0C604745F6452CC0F6BD
:1000C0000E0C604748F2B35CC0F60C0C604744F677
:1000D0004D3CC0F60D0C604745F6DF1CC0F60D0C1C
:1000E000604743F6816CC0F60D0C60474DF6593CF5
:1000F000C0F60C0C60474CF63D5CC0F60C0C60473B
:1001000044F66D7CC0F6020C604746F2EF3CC0F648
:100110000D0C60474FF61F4CC0F60C0C60474DF2BB
:10012000A91CC0F60C0C604741F2CF5CC0F60E0C67
:10013000604741F21D6CC0F60E0C604745F25B6CE7
:10014000C0F6020C60474DF2C95CC0F6020C604775
:100150004AF6052CC0F6020C60474AF60D2CC0F694
:10016000020C604746F2A74CC0F6020C604746F20C
:10017000EF4CC0F6020C604746F2C31CC0F6020CFE
:10018000604746F2C10CC0F6020C604748F2752C7D
:10019000C0F6020C604748F2593CC0F6020C6047BA
:1001A00048F2514CC0F6020C60474CF2215CC0F69C
:1001B0000C0C604748F27D5CC0F6020C604745F6C7
:1001C000E76CC0F6020C604748F2974CC0F6020C90
:1001D000604748F2AD5CC0F6020C604745F2A30CE4
:1001E000C0F6020C604740F2812CC0F6020C60475A
:1001F00040F2852CC0F6020C60474CF6916CC0F6BC
:100200000C0C60474DF6E50CC0F60C0C60474DF247
:10021000455CC0F60C0C60472DE9F04591B00446F2
:100220000E46D4F87C0EB04228D100200F901090DA
:10023000D4F86C1ED1F8BC2104F5247151F82200C9
:100240000FA900F0B5FC0FA904F5657000F051FD91
:10025000012809D141F288306EA370A272A10090EA
:100260002046FFF7DFFE08E041F2883069A370A264
:100270006DA100902046FFF7D5FEC8E0D4F8840EAB
:10028000B04235D10127D4F8880E28B1D4F8880EB1
:10029000B0F8BC01401C87B2D4F8780E00F5DE75CA
:1002A0004FF48070FFF7C3FE804641462846FFF7B3
:1002B000C3FE4046FFF7C5FE8246534642463946D6
:1002C00004F5657000F02AFF4046FFF7BFFE0223E9
:1002D0005AA2394604F5657000F020FFD4F8781E64
:1002E00001F5DE727321D4F8740EFFF7B4FE8EE0D0
:1002F000D4F8800EB042C0D1D4F88C02022814D1B8
:10030000D4F8700E00F5DE7104F5657000F06FFF33
:10031000D4F8700ED0F8981188470020C4F8700EF9
:1003200004F5657000F080FF13E0D4F88C0201281A
:100330000FD104F66C642068D0F89811884700202B
:1003400020602069D0F89811884700202061A4F629
:100350006C64012104F5657000F015FFD4F8800E7F
:10036000D0F8981188470020C4F8800E322120462A
:10037000FFF776FEA568E768C820A5F10A03052205
:10038000114600902046FFF770FEC4F8740E282036
:10039000A5F1A003CD22052100902046FFF76AFEBB
:1003A000C4F8780E20222649794409A8FFF767FE91
:1003B00009A80490801D05900CA80690801D079048
:1003C0000FA8089028206421CD22A5F19B03CDE938
:1003D00000210290052204A92046FFF755FEC4F82B
:1003E000880E19203221A5F13702D223CDE9001061
:1003F00000212046FFF74DFEC4F8840E11A1D4F869
:10040000840EFFF74BFE2046FFF74DFE00BF11B0F4
:10041000BDE8F085C8B7B6A800000000C1ACBDD3E8
:10042000B3C9B9A600000000CCE1CABE00000000BC
:10043000C1ACBDD3CAA7B0DC000000000D0A0000AB
:100440004C150000B7A2CBCD000000002DE9F04113
:1004500006460C4601F080F907464FF000080025DB
:1004600020680A2843D2DFE800F04209050D423037
:100470004222422C304600F0C1F839E0304600F00C
:100480003DF835E0E568287C00F0010000B900BFC8
:10049000287C00F0080020B13046D6F89811884733
:1004A00026E0286910B13046FFF7FDFD20E0D4F8C2
:1004B0000C80D8F80800032800D100E000BF00BF7E
:1004C00016E0304600F028F812E0E068012802D07B
:1004D000022809D100E008E02069012803D1304654
:1004E0006168FFF799FE00E000BF00BF00E000BFB9
:1004F00000BF384601F058F9BDE8F0812DE9F04120
:10050000044600250026A768D4F80C802046FFF793
:10051000CFFDBDE8F08100002DE9F84F064600BF91
:1005200006F5657000F007FC0028F9D14FF48070E3
:10053000FFF77DFD04460025002756E04FF0000838
:10054000394606F5657000F071FC8046B8F1000F81
:100550004AD038E00020605500BF11E0691E091A3A
:100560000DD4691E091A615C0D2904D0691E091A8F
:10057000615C0A2903D10022691E091A6254401CD9
:100580000328EBDBD6F8740EE8B14FF48070FFF768
:100590004EFD8246B8F8062017A15046FFF78DFDA4
:1005A0005046FFF74EFD00EB0A0B59462046FFF779
:1005B00089FD52467221D6F8740EFFF74CFD504665
:1005C000FFF744FD00BF0A200090B8F8061064232E
:1005D000224606F5657000F0AEFC05460DB101201F
:1005E00000E000200028B5D17F1C052FA6DB2046A7
:1005F000FFF72CFDBDE8F88F25643A002DE9FE4F8A
:100600000446A668E56804F5657000F0ACFC04F5E6
:10061000657000F0D9FC70B941F2883066A368A219
:100620006CA100902046FFF7FDFC2046D4F89811FD
:100630008847BDE8FE8F94F8880231287DD10120DB
:10064000C4F88C0204F5657000F0B6FD2346634AD9
:100650007A4463A12046FFF73AFD06EB46082F4691
:100660002D205A21CDE90010E81705EB907083107A
:100670004FEAE87008EB9070821000212046FFF7E7
:1006800008FDC4F87C0E5BA1D4F87C0EFFF706FDD4
:1006900006EB460805EB45072D208221CDE9001029
:1006A000F81707EB907083104FEAE87008EB907032
:1006B000821000212046FFF7ECFCC4F8800E4FA109
:1006C000D4F8800EFFF7EAFC06EB4600052190FB0C
:1006D000F1FA2F464FEA45084FEAE87008EB9070B0
:1006E0008010E91705EB9171891014230022CDE9E0
:1006F000001A029004F524712046FFF7C5FCC4F8E7
:100700006C0E002713E004F5247050F82780803029
:1007100050F82700007818B104F5447050F827808D
:1007200000224146D4F86C0EFFF7D6FC7F1CD4F8AB
:100730009003B842E7DC39E0FFE794F888023228FA
:1007400034D10220C4F88C02B04605EB45072D20B9
:100750008221CDE90010F81707EB9070831006EBAB
:10076000D870421000212046FFF793FCC4F8800E99
:1007700022A1D4F8800EFFF791FCB2462F46B34673
:10078000A846E81705EB90708010009006EBDB7030
:100790004310E81705EB90708210F01706EB90708D
:1007A00081102046FFF766FCC4F8700E2046FFF764
:1007B0007AFC00BF3DE70000C8B7B6A80000000003
:1007C000C0B6D1C0C4A3BFE9B8B4CEBBCAA7B0DC21
:1007D000A3A10000B4EDCEF300000000F90F00006B
:1007E000D5FDD4DAC9A8C3E8C0B6D1C0B4D3BBFA2A
:1007F0002E2E2E00C1ACBDD300000000CFC2D2BB54
:10080000B2BD00007CB50446002610A011A313A2BF
:1008100015A100902046FFF764FC08B9312600E0DE
:100820003226D4E9020100231A46CDE90001194617
:10083000204600F01DF8054685F888622846FFF737
:1008400055FC2846FFF757FC28467CBDB4D3BBFABD
:1008500000000000D6F7BBFA00000000C7EBD1A1F2
:10086000D4F1BDC7C9AB0000CCE1CABE0000000096
:100870002DE9FE4F07460E4690469A46DDF830B009
:100880000EB9264E7E4440F68C60FFF7D0FB04463E
:10089000002C3AD040F68C6200212046FFF730FC55
:1008A0000D98434632463946CDE900AB02902046CA
:1008B000FFF72BFC20B92046FFF7C8FB002424E0FB
:1008C00017A060610120C4F82C0119487844C4F8CD
:1008D00098010020A063174860631020FFF71AFCFE
:1008E000C4F8840200250EE01420FFF7A0FB04F5F5
:1008F000247141F825001420FFF799FB04F5447199
:1009000041F825006D1C202DEEDB00F069FF0A4840
:10091000484404602046BDE8FE8F0000C5FBFFFF91
:1009200057494E5F43686174537472756374000075
:100930006D000000ACC1D7000800000070B504468F
:1009400000F00AFF064600250CE004F5247151F87A
:100950002500FFF77BFB04F5447151F82500FFF7F4
:1009600075FB6D1C202DF0DB04F5657000F02CFB91
:10097000D4F88402FFF7CEFB2046FFF7D0FB00201F
:1009800004494944086000F015FF304600F00CFFB0
:1009900070BD00000800000070B5054600F0DCFEE8
:1009A000044607484844006820B1054848440068A8
:1009B000FFF7C4FF204600F0F7FE002070BD0000E6
:1009C000080000000146FF20302904DB392902DC41
:1009D000A1F13002D0B2412904DB462902DCA1F1A9
:1009E0003702D0B2704710B500F062FC002010BD95
:1009F0002DE9F04D04460E4617469846DDE908AB52
:100A00002078FF2803D04FF0FF30BDE8F08D701E36
:100A1000205CFC2802D04FF0FF30F6E74FF0FF35A6
:100A2000721EFB21601C00F002FE0546681C30B3FC
:100A3000BAF1000F02D0FB208AF80000B8F1000FD5
:100A400005D02946601C00F011FFC8F800000FB166
:100A5000601C38600A9840B1F21E511B621C2A4487
:100A6000501C00F003FF0A990860BBF1000F04D08E
:100A7000601C2844401CCBF800000020C5E7721E13
:100A8000FA21601C00F0D3FD0546681C30B3BAF1B2
:100A9000000F02D0FA208AF80000B8F1000F05D04C
:100AA0002946601C00F0E2FEC8F800000FB1601C8F
:100AB00038600A9840B1F21E511B621C2A44501C37
:100AC00000F0D4FE0A990860BBF1000F04D0601C4E
:100AD0002844401CCBF80000002096E74FF0FF3080
:100AE00093E7F8B5054600200090002400260EE0AC
:100AF0009DF80000FF2800D101261EB19DF80000DE
:100B00002855641C9DF80000FC2800D104E06846CC
:100B100000F0E2FB0028EBD000BF9DF80000FC28AD
:100B200001D12046F8BD4FF0FF30FBE710B500F0D3
:100B3000DDFB002010BD70B505460E46002403E025
:100B4000285D00F047FC641CB442F9DB002070BD56
:100B50002DE9F04105460C461646FF20134949444D
:100B6000087008464570FD20887004B14EB9FC201D
:100B70000E494944C87004210C484844FFF7DBFF84
:100B800011E0324609494944C91C204600F035FDB0
:100B90000746FC21F81C054A4A441154391D1046E9
:100BA000FFF7C9FF00BF0020BDE8F0814C02000044
:100BB0002DE9F04706460F463546B8460024A246C2
:100BC00017E02878FFF7FEFE8246BAF1FF0F0FD03C
:100BD00008EB6400007804F0010109B1002100E095
:100BE00004210AFA01F1084308EB64010870641C4F
:100BF0006D1C28780028E4D12046BDE8F08730B588
:100C000002460B460BB9002030BD002418E0C4EBAF
:100C1000041000EBC00502F1080000EB8501C88854
:100C200068B9D2F8B45A0D60B2F8B80A8880CB809F
:100C3000012088605068401C50600120E4E7641C7B
:100C4000052CE4DB0020DFE72DE9F04D04468B4660
:100C500017469846DDF824A000BFD4F8B00A012852
:100C60000EDAD4F8B00A00EBC00101EB001104F673
:100C700094200D18D4F8B00A401CC4F8B00A23E040
:100C8000D4F8B00A401E00EBC00101EB001104F6DD
:100C900094200D18002612E0721C02EBC20303EB35
:100CA000021304F69422991806EBC60202EB06130F
:100CB00004F6942298181922FFF736FA761CD4F815
:100CC000B00A401EB042E7DC2F703A465946681C15
:100CD000FFF72AFA781C054485F800806D1C85F81A
:100CE00000A05246681C0899FFF71EFA0120BDE8D3
:100CF000F08DF8B504460D4604F6BA2600200090A3
:100D0000062229462120FFF723FF6A463146204666
:100D100000F0A4F801280CD13078012809D104F59D
:100D200028602968C4F8B41AA988A4F8B81A012060
:100D3000F8BD0020FCE730B5A1B0054600246421D1
:100D400008A8FFF7F6F908A8FFF7CBFE0446601CD9
:100D500028B908A8FFF7F2F9002021B030BD002023
:100D60000790069005900490039006A807A903AA8F
:100D700004ABCDE90021029005AA214608A8FFF79F
:100D800037FE401C20B908A8FFF7D8F90020E4E797
:100D90009DF80C00FB280BD1DDE90610CDE9000120
:100DA0009DF80C302846DDE90421FFF74DFF1AE0DD
:100DB0009DF80C00FA2816D105980078012806D174
:100DC000079842880188284600F0E9F80BE005986A
:100DD0000078022807D10698831E07980188821C94
:100DE000284600F020F90120B7E710B502460B466F
:100DF0000BB9002010BD002114E0C1EB011000EB85
:100E0000C00402F1080000EB8400C088984208D1B9
:100E1000C1EB011000EBC00402F1080000EB8400FC
:100E2000E8E7491C0529E8DB0020E3E7024605293D
:100E300012DAC1EB011000EBC00302F1080000EB75
:100E40008300C08840B1C1EB011000EBC00302F188
:100E5000080000EB830070470020FCE77CB50646E5
:100E60000C46154600BF3046FFF765FF00231A46C3
:100E700019463046CDE9004500F004F80028F2D0CC
:100E800001207CBD2DE9F04D05460F4690469A465F
:100E9000DDF820B0D5F8B00A00284AD005F6942431
:100EA00027B12278611C3846FFF73EF9B8F1000FF0
:100EB00002D02078C8F80000BAF1000F04D02078E2
:100EC000401C205C8AF80000BBF1000F08D020789D
:100ED000801C225C2078C01C01195846FFF724F9B9
:100EE000099820B12078801C215C099801600026B7
:100EF00012E0721C02EBC20303EB021305F694220C
:100F0000991806EBC60202EB061305F69422981810
:100F10001922FFF709F9761CD5F8B00A401EB04235
:100F2000E7DCD5F8B00A401EC5F8B00A0120BDE8DC
:100F3000F08D0020FBE72DE9F04707468846144670
:100F40001D46DDF820A041463846FFF74EFF064615
:100F50003EB153462A462146304600F00EFBBDE81E
:100F6000F0870020FBE770B50446FFF7DFFD69203E
:100F7000207000206060C4F8B00A00250AE0C5EBCC
:100F8000051101EBC10204F1080101EB820000F040
:100F9000E7FA6D1C052DF2DBFFF725FD70BD70B57E
:100FA00005460E461446012C04D131462846FFF76B
:100FB00026FE07E024B93146284600F050F901E04A
:100FC000002070BD0120FCE7FEB5044604F6BA25FA
:100FD00000200290642600BF002211460320FFF784
:100FE000B7FD0220FFF7AFF82046FFF7A4FE02A8E6
:100FF00000231A461946CDE900502046FFF742FF6C
:101000000298012809D12878012806D16420FFF729
:101010009AF8FFF7E8FC0120FEBD3000A6F10106BA
:10102000DAD100BFF8E72DE9F041074688461446BB
:101030001D4641463846FFF7D8FE064636B12A46D9
:101040002146304600F0C2FABDE8F0810020FBE7FF
:101050002DE9F84307460D46144607F6BA26002048
:1010600000902060002211462320FFF771FD40F61A
:10107000AC50FFF768F850E06A4631463846FFF753
:10108000EDFE012847D10098012806D130780128CB
:1010900001D1BDE8F8830020FBE7009807283CDB7E
:1010A000206800EBC00000EB40002844316801607C
:1010B000B1888180B07940B2216801EBC10101EBB8
:1010C0004101294488710098072818DD0098A0F193
:1010D0000708216801EBC10101EB41012944C81D4A
:1010E0004246F11DFFF720F80021206800EBC00008
:1010F00000EB40002844C01D00F8081007E0002065
:10110000216801EBC10101EB41012944C87120684C
:10111000401C206001E00020BBE7ADE72DE9F84569
:1011200082460F4690461C460AF6BA2500200090DB
:10113000002624E02F7038126870142C01DD14266C
:1011400000E0264632464146A81CFEF7EDFFB21CE1
:1011500029460720FFF7FCFC6A4629465046FFF760
:101160007DFE012807D12878012802D12CB9BDE8DD
:10117000F8850020FBE70020F9E7A41BB044002C11
:10118000D8D10020F3E733B581B0054605F6BA247F
:1011900000200090012202A90620FFF7D9FC6A4630
:1011A00021462846FFF75AFE012803D1207801285E
:1011B00000D13EBD0020FCE738B5044604F6BA2550
:1011C00000200090002211462020FFF7C1FC6A4653
:1011D00029462046FFF742FE012806D1287801283B
:1011E00003D168202070012038BD0020FCE7F8B54D
:1011F00004460D4604F6BA26002000902846FEF765
:1012000020FF07463A4629460120FFF7A1FC6A461F
:1012100031462046FFF722FE012803D1307801280D
:1012200000D1F8BD0020FCE738B5044604F6BA2525
:1012300000200090002211461020FFF789FC6A462A
:1012400029462046FFF70AFE012806D12878012802
:1012500003D173202070012038BD0020FCE72DE968
:10126000F04105460E4616B90020BDE8F081002782
:1012700019E0C7EB071000EBC00105F1080000EB17
:101280008104E088B0420DD10020E080A0602060A1
:10129000A08004F10C0000F0AFF86868401E6860A0
:1012A0000120E2E77F1C052FE3DB0020DDE70000E3
:1012B00010B5FEF74DFF044600200649494448603A
:1012C0008860C860086148612046FEF746FF00203C
:1012D00010BD00003400000010B50446214602484D
:1012E000484400F0B0F810BD3400000000B587B0ED
:1012F00001210846FEF736FF01211020FEF737FFD7
:10130000072209212F48FEF737FF07220A212D481F
:10131000FEF732FF00208DF81A0001208DF81B0027
:1013200002208DF818000002059002208DF81900A7
:1013300005A92448FEF725FF00208DF81A00022099
:101340008DF818004002059005A91E48FEF719FF08
:101350001D48FEF71BFF4FF4E13001900020ADF86F
:101360000800ADF80A00ADF80C00ADF810000C2034
:10137000ADF80E0001A91448FEF70DFF0121124837
:10138000FEF70EFF114979442520FEF70EFF0122DA
:1013900040F225510C48FEF70DFF25208DF8000086
:1013A00000208DF8010001208DF802008DF8030067
:1013B0006846FEF704FF4FF4007005494944086091
:1013C00007B000BD000002400010014017050000FA
:1013D0003400000010B5044621460648FEF7F4FE2E
:1013E00000BF80210348FEF7F4FE0028F9D000205A
:1013F00010BD0000001001400146002048608860D8
:10140000C860704730B502460B46916854680BE0DF
:1014100002F11000405C984201D1012030BD491C0E
:101420001068884200DC00212000A4F10104EFD103
:1014300000BFF3E710B504464FF40070206020466B
:10144000FFF7DAFF10BD2DE9F04104460D464FF0DD
:10145000FF36FEF77DFE07462069C8B16068B8B167
:1014600004F11800A168405C28706068401E60604C
:101470002878FC2802D12069401E2061A068401C09
:10148000A0602168A068884201DB0020A0600026DF
:101490003846FEF762FE3046BDE8F08102465068ED
:1014A00090B102F110009368C05C08705068401E53
:1014B00050609068401C906013689068984201DB0F
:1014C00000209060012070470020FCE72DE9F041EA
:1014D00004460D464FF0FF36FEF73AFE0746FF2D55
:1014E00001D101206061D4E90010884219DA6069F5
:1014F000B8B104F11800E16845546068401C6060B0
:10150000FC2D04D12069401C206100206061E0684E
:10151000401CE0602168E068884201DB0020E06058
:1015200000263846FEF719FE3046BDE8F081024637
:10153000D2E90030984211DA02F11000D368C154A8
:101540005068401C5060D068401CD0601368D06860
:10155000984201DB0020D060012070470020FCE7AA
:1015600010B504460020E080A0602060A08004F157
:101570000C00FFF75FFF012010BD2DE9F843054681
:10158000884616461F46394605F10C00FFF73AFF1C
:1015900010B90020BDE8F88300240020009014E07A
:1015A000694605F10C00FFF779FF08B92046F1E71D
:1015B0002EB19DF8000008F80400761E641C9DF80A
:1015C0000000B84201D12046E4E7E9E72DE9F04107
:1015D00005460E461746002409E0315D05F10C0072
:1015E000FFF7A5FF10B92046BDE8F081641C380064
:1015F000A7F10107F1D12046F6E730B503460C46C6
:101600000FE01878F02804DA18780870491C5B1C81
:1016100007E0F0200870491C1878F0380870491C61
:101620005B1C1000A2F10102EBD1081B30BD10B50C
:101630000346002004E01C5C8C4200D110BD401C1D
:101640009042F8DB4FF0FF30F8E700002DE9FF4D46
:10165000074600F081F883463E464FF45870FEF787
:10166000E6FC054606F564722946101DFFF7F0FCFE
:10167000002455E006F5247050F8248004EBC400E3
:1016800000EB40002844407904EBC40101EB410128
:101690002944097904EBC40202EB42022A44D278BD
:1016A00004EBC40303EB43032B449B78CDE90032E6
:1016B000CDE9021004EBC40000EB4000284443785D
:1016C00004EBC40000EB40002A5C1CA14046FEF77E
:1016D000F4FC04EBC40000EB40002844C079C0B126
:1016E00006F5447050F8248004EBC40101EB41017D
:1016F0002944C81DFEF7A5FC00F1010A04EBC40053
:1017000000EB40002844C11D52464046FEF766FDEE
:1017100005E0002106F5447050F824000170641CB7
:10172000D6F89003A042A5DC2846FEF78FFC584669
:1017300000F03AF8002004B0BDE8F08D25303258B2
:10174000253032582530325825303258253032581D
:10175000253032580000000010B5FEF744FD044665
:10176000034878440068FEF743FD204610BD0000A2
:101770008E01000070B50446FEF735FD054629468A
:1017800006487844FEF74CFC054848440460054888
:101790007844034949440968486170BD6E010000FE
:1017A0000400000005F2FFFF10B504462046FEF7D6
:1017B0001FFD10BD09484844006868B10748484407
:1017C0000068806940B10548484400688069401E4F
:1017D000024949440968886170470000040000001C
:1017E00006484844006840B104484844006880699D
:1017F000401C0249494409688861704704000000A0
:1018000070B505462846FFF7B5FFFFF7E9FF00244E
:1018100011A10020FEF7F1FC04460CB9012000E004
:10182000002068B10FA10020FEF7E7FC0646304615
:10183000FEF7E8FF044608A12046FEF7E3FC07E0B8
:101840002146D4F84001FEF7E2FC2046FEF753FCA7
:10185000FFF7B0FF002070BD626C652063686174A3
:1018600000000000686F6D650000000030B50346A1
:101870000C4619461A460FE00878F02805DA087871
:101880001070521C491C641E06E008784D782844EC
:101890001070521C891CA41E002CEDD1D01A30BD32
:1018A00070B5FFF759FF044600250F48008800F087
:1018B000200078B10C488088C5B229460B484844BE
:1018C000FFF704FE0A4848440068401C08494944A0
:1018D000086005E004480088C5B203488088C5B2A6
:1018E0002046FFF761FF70BD00100140340000008A
:1018F0001000000000000000CDA8B5C03100CDA848
:10190000B5C03200CDA8B5C03300CDA8B5C03400F5
:10191000CDA8B5C0350000000000000000000000A8
:0C192000000000000100000000000000BA
:0400000500001801DE
:00000001FF
